S01400006F7064726163687420342E312E7372656308
S113000045C0000058C0000056C0000054C00000A5
S113001052C0000050C000004EC000004CC00000A0
S11300204AC00000DFC0000046C0000044C0000019
S113003042C0000040C000003EC000003CC00000C0
S11300403AC0000038C0000036C0000034C00000D0
S113005032C0000030C000002EC000002CC00000E0
S11300602AC0000028C0000026C0000024C00000F0
S113007022C0000020C000001EC000001CC0000000
S11300801AC0000018C0000016C0000011241FBED2
S1130090CFEFD0E1DEBFCDBF11E0A0E0B1E0E2E3FD
S11300A0F2E000E00BBF02C007900D92AC30B10744
S11300B0D9F7A2D0BCC0A4CF9BB321E030E002C0EA
S11300C0220F331F8A95E2F7292B2BBB08959BB38C
S11300D021E030E002C0220F331F8A95E2F7209519
S11300E029232BBB089586E090E0E6DF89EF90E0BA
S11300F00197F1F700C0000086E090E0E8DF89EFA7
S113010090E00197F1F700C000000895CF93C82F45
S113011085BB84E090E0D0DFE6DFC295C07FC5BB3D
S113012084E090E0C9DFDFDFCF910895CF93C82F3B
S113013085BB84E090E0CBDFD6DFC295C07FC5BB32
S113014084E090E0C4DFCFDFCF91089581E0EEDF5B
S113015083EF91E00197F1F700C0000080E8E6CF5B
S11301600895CF938FEF84BB85BB8ABB15BA1BBAA6
S1130170C0E2C5BBB8DFC5BBB6DF80E885BBB3DF73
S113018015BAB1DF80EF85BBAEDF15BAACDF80E610
S113019085BBA9DF82E0CADFA6DFCF910895CF93A4
S11301A0DF93EC0102C0B2DF219688818111FBCF7D
S11301B0DF91CF9108958EE1B9CF089520E030E02A
S11301C008C0E3ECF9E03197F1F700C000002F5FBD
S11301D03F4F28173907ACF3089580EE87B986E8B6
S11301E086B908951F920F920FB60F9211240F90A3
S11301F00FBE0F901F901895109261008FEF82B977
S1130200ECDFAFDFA3DFD7DFD6DF80E091E0C7DF2D
S113021087EA91E60197F1F700C0000086B1806497
S113022086B985B183B98AE090E0C8DFF7CFF89446
S1050230FFCFFA
S10F02324D4F4F4F4F4F4F4F4F4F0000A8
S9030000FC
